:020000040000FA
:100000000C9462000C948A000C948A000C948A0070
:100010000C948A000C948A000C948A000C948A0038
:100020000C948A000C948A000C948A000C948A0028
:100030000C948A000C948A000C948A000C948A0018
:100040000C9418030C948A000C94E6020C94C002E1
:100050000C948A000C948A000C948A000C948A00F8
:100060000C948A000C948A000000000024002700F1
:100070002A0000000000250028002B0000000008D6
:10008000000201000003040700000000000000005F
:1000900000000000230026002900040404040404D6
:1000A0000404020202020202030303030303010227
:1000B00004081020408001020408102001020408F6
:1000C00010205E0511241FBECFEFD8E0DEBFCDBFEC
:1000D00011E0A0E0B1E0E6E9FEE002C005900D927B
:1000E000A634B107D9F721E0A6E4B1E001C01D9222
:1000F000A13FB207E1F710E0C2E6D0E004C02197CB
:10010000FE010E944307C136D107C9F70E94A70329
:100110000C9449070C940000AF92BF92CF92DF92EB
:10012000EF92FF920F931F93CF93DF936C017B01AC
:100130008B01040F151FEB015E01AE18BF08C0173D
:10014000D10759F06991D601ED91FC910190F081B0
:10015000E02DC6010995892B79F7C501DF91CF9173
:100160001F910F91FF90EF90DF90CF90BF90AF90D5
:100170000895FC01538D448D252F30E0842F90E0AD
:10018000821B930B541710F0CF9608950197089592
:10019000FC01918D828D981761F0A28DAE0FBF2F5B
:1001A000B11D5D968C91928D9F5F9F73928F90E0B1
:1001B00008958FEF9FEF0895FC01918D828D981720
:1001C00031F0828DE80FF11D858D90E008958FEF5D
:1001D0009FEF0895FC01918D228D892F90E0805C26
:1001E0009F4F821B91098F739927089584E591E0B1
:1001F0000E94EA0021E0892B09F420E0822F089573
:1002000080E090E0892B29F00E94F60081110C9487
:1002100000000895FC01A48DA80FB92FB11DA35AA9
:10022000BF4F2C91848D90E001968F739927848F16
:10023000A689B7892C93A089B1898C918370806439
:100240008C93938D848D981306C00288F389E02DDA
:1002500080818F7D80830895EF92FF920F931F938B
:10026000CF93DF93EC0181E0888F9B8D8C8D981369
:100270001AC0E889F989808185FF15C09FB7F89475
:10028000EE89FF896083E889F989808183708064C1
:1002900080839FBF81E090E0DF91CF911F910F910C
:1002A000FF90EF900895F62E0B8D10E00F5F1F4F1B
:1002B0000F731127E02E8C8D8E110CC00FB607FC2A
:1002C000FACFE889F989808185FFF5CFCE010E94B8
:1002D0000A01F1CFEB8DEC0FFD2FF11DE35AFF4F1B
:1002E000F0829FB7F8940B8FEA89FB898081806246
:1002F000CFCFCF93DF93EC01888D8823B9F0AA8903
:10030000BB89E889F9898C9185FD03C0808186FDD0
:100310000DC00FB607FCF7CF8C9185FFF2CF80811F
:1003200085FFEDCFCE010E940A01E9CFDF91CF9189
:100330000895833081F028F4813099F08230A9F05B
:1003400008958730A9F08830C9F08430B1F48091E5
:1003500080008F7D03C0809180008F778093800024
:10036000089584B58F7784BD089584B58F7DFBCFC4
:100370008091B0008F778093B00008958091B00095
:100380008F7DF9CFCF93DF93282F30E0F901E45828
:10039000FF4F8491F901E255FF4FD491F901E656E0
:1003A000FF4FC491CC23A1F081110E949901EC2F41
:1003B000F0E0EE0FFF1FE057FF4FA591B491EC91D5
:1003C000ED2381E090E009F480E0DF91CF91089582
:1003D00080E090E0FACF1F93CF93DF93282F30E097
:1003E000F901E458FF4F8491F901E255FF4FD49190
:1003F000F901E656FF4FC491CC23A9F0162F8111C5
:100400000E949901EC2FF0E0EE0FFF1FEE58FF4F16
:10041000A591B4918FB7F894EC91111108C0D095C3
:10042000DE23DC938FBFDF91CF911F910895DE2BE8
:10043000F8CFCF93DF9390E0FC01E255FF4F24917A
:1004400086569F4FFC0184918823D1F090E0880F5D
:10045000991FFC01E859FF4FA591B491FC01EE589A
:10046000FF4FC591D49161110EC09FB7F8948C9144
:10047000E22FE0958E238C932881E223E8839FBFAF
:10048000DF91CF9108958FB7F894EC91E22BEC9324
:100490008FBFF6CF3FB7F89480914B0190914C01FC
:1004A000A0914D01B0914E0126B5A89B05C02F3FEC
:1004B00019F00196A11DB11D3FBFBA2FA92F982F8A
:1004C0008827BC01CD01620F711D811D911D42E085
:1004D000660F771F881F991F4A95D1F70895FC0171
:1004E00001900020E9F73197AF01481B590BBC017F
:1004F00084E591E00C948C008F929F92AF92BF9212
:100500000F931F93CF93DF93CDB7DEB7A1970FB6AD
:10051000F894DEBF0FBECDBF19A2423008F44AE006
:100520008E010F5D1F4F842E912CB12CA12CA501A3
:1005300094010E942107E62FB901CA01EA30F4F4C0
:10054000E05DD801EE938D01232B242B252B79F729
:1005500090E080E0109719F0CD010E946F02A19603
:100560000FB6F894DEBF0FBECDBFDF91CF911F91C4
:100570000F91BF90AF909F908F900895E95CE1CF6D
:100580001F920F920FB60F9211242F933F934F9308
:100590005F936F937F938F939F93AF93BF93EF93EB
:1005A000FF9384E591E00E940A01FF91EF91BF91D2
:1005B000AF919F918F917F916F915F914F913F91FB
:1005C0002F910F900FBE0F901F9018951F920F92B2
:1005D0000FB60F9211242F938F939F93EF93FF9356
:1005E000E0916401F09165018081E0916A01F091F0
:1005F0006B0182FD1BC0908180916D018F5F8F73B5
:1006000020916E01821741F0E0916D01F0E0EC5A0B
:10061000FE4F958F80936D01FF91EF919F918F9188
:100620002F910F900FBE0F901F9018958081F4CFDF
:100630001F920F920FB60F9211242F933F938F9317
:100640009F93AF93BF938091470190914801A091F0
:100650004901B0914A013091460123E0230F2D3723
:1006600058F50196A11DB11D2093460180934701C5
:1006700090934801A0934901B0934A0180914B01A6
:1006800090914C01A0914D01B0914E010196A11D98
:10069000B11D80934B0190934C01A0934D01B093F9
:1006A0004E01BF91AF919F918F913F912F910F90EC
:1006B0000FBE0F901F90189526E8230F0296A11DDC
:1006C000B11DD2CFCF92DF92EF92FF920F931F9383
:1006D000E82FF92F05C0015011092109310961F1F5
:1006E000908196239417B9F305C00150110921098F
:1006F000310911F1908196239413F7CFC12CD12C9D
:10070000E12CF12C0AC08FEFC81AD80AE80AF80ABF
:100710000C151D052E053F0579F080818623841771
:1007200091F36C2D7D2D8E2D9F2D1F910F91FF909C
:10073000EF90DF90CF90089560E070E080E090E06F
:100740001F910F91FF90EF90DF90CF9008957894D4
:1007500084B5826084BD84B5816084BD85B58260C6
:1007600085BD85B5816085BD80916E008160809377
:100770006E001092810080918100826080938100E0
:1007800080918100816080938100809180008160F0
:10079000809380008091B10084608093B10080914B
:1007A000B00081608093B00080917A008460809373
:1007B0007A0080917A00826080937A0080917A003A
:1007C000816080937A0080917A00806880937A00BB
:1007D0001092C10060E082E00E94190260E083E0B4
:1007E0000E94190261E084E00E94190261E085E044
:1007F0000E941902E0916401F091650182E080831A
:10080000E0916001F09161011082E0916201F0914C
:1008100063018FEC808310926C01E0916801F0918C
:10082000690186E08083E0916601F0916701808133
:1008300080618083E0916601F0916701808188602A
:100840008083E0916601F0916701808180688083F8
:10085000E0916601F091670180818F7D80834BE993
:10086000242E312C2BE3E22EFF24F39430E0C32E10
:1008700030E0D32E82E00E94C201019709F012C13C
:1008800060E084E00E94EB0183E090E00197F1F7E3
:1008900061E084E00E94EB018BE490E00197F1F7C6
:1008A00060E084E00E94EB01E1EBF0E06491EDE9AF
:1008B000F0E08491E82FF0E0EE0FFF1FE057FF4FCC
:1008C0008591949100E412E42FE030E0462F0E94DD
:1008D0006203611571058105910529F06F5F7F4FF6
:1008E0008F4F9F4F9F700E94020620E034E244E742
:1008F00059E40E94900520E030E04AEA53E40E9467
:10090000B40620E030E040E05FE30E94B40620E05F
:1009100030E048EC52E40E94B40620E030E040EFC2
:1009200051E40E948B0587FFBDC060E085E00E9416
:10093000EB010E944A024B015C018EE1482E512CD2
:10094000612C712C0E944A02681979098A099B0955
:10095000683E734081059105A8F3F1E04F1A5108F4
:100960006108710828EE820E23E0921EA11CB11CC2
:10097000411451046104710429F761E085E00E948B
:10098000EB01C1010197F1F760E085E00E941902D7
:1009900085E00E94C2010197D9F3C7010197F1F7E1
:1009A00085E00E94C201892BD9F3C7010197F1F7B5
:1009B0000FE411E0C8E0D0E0712C85E00E94C20194
:1009C000892BE1F485E00E94C201892BD9F383E7EA
:1009D00090E00197F1F785E00E94C2018130910516
:1009E00041F49E012150310901C0880F2A95EAF790
:1009F000782A85E00E94C2010197D9F32197E9F690
:100A0000F80171928F0184E591E08E179F0791F6AE
:100A100061E085E00E94190261E085E00E94EB013F
:100A200082E191E00E946F0260914F0170E090E0DE
:100A300080E04AE00E947C026EE284E591E00E9440
:100A40002C016091500170E090E080E04AE00E944B
:100A50007C0285E291E00E946F0288E291E00E94B0
:100A60006F028BE291E00E946F026091510170E091
:100A700090E080E04AE00E947C026EE284E591E032
:100A80000E942C016091520170E090E080E04AE009
:100A90000E947C0282E491E00E946F0288E291E071
:100AA0000E946F02C114D10409F4E4CE0E94F60042
:100AB000882309F4D7CE0E940000D4CEE4E5F1E00B
:100AC0001382128288EE93E0A0E0B0E084839583E5
:100AD000A683B78384E091E09183808385EC90E0E6
:100AE0009587848784EC90E09787868780EC90E0F8
:100AF000918B808B81EC90E0938B828B82EC90E0E9
:100B0000958B848B86EC90E0978B868B118E128E62
:100B1000138E148E08950E943F0608F481E0089514
:100B20000E94A4050C947A060E94730658F00E9455
:100B30006C0640F029F45F3F29F00C9463065111D4
:100B40000C94AE060C9469060E948B0668F39923F8
:100B5000B1F3552391F3951B550BBB27AA276217B9
:100B60007307840738F09F5F5F4F220F331F441FC6
:100B7000AA1FA9F335D00E2E3AF0E0E832D09150FA
:100B80005040E695001CCAF72BD0FE2F29D0660FE7
:100B9000771F881FBB1F261737074807AB07B0E82A
:100BA00009F0BB0B802DBF01FF2793585F4F3AF030
:100BB0009E3F510578F00C9463060C94AE065F3F9F
:100BC000E4F3983ED4F3869577956795B795F795B6
:100BD0009F5FC9F7880F911D9695879597F908959E
:100BE000E1E0660F771F881FBB1F6217730784073A
:100BF000BA0720F0621B730B840BBA0BEE1F88F749
:100C0000E0950895E89409C097FB3EF4909580958F
:100C1000709561957F4F8F4F9F4F9923A9F0F92FC2
:100C200096E9BB279395F695879577956795B79540
:100C3000F111F8CFFAF4BB0F11F460FF1BC06F5F26
:100C40007F4F8F4F9F4F16C0882311F096E911C038
:100C5000772321F09EE8872F762F05C0662371F059
:100C600096E8862F70E060E02AF09A95660F771F6D
:100C7000881FDAF7880F9695879597F90895990F49
:100C80000008550FAA0BE0E8FEEF16161706E80756
:100C9000F907C0F012161306E407F50798F0621B77
:100CA000730B840B950B39F40A2661F0232B242B4C
:100CB000252B21F408950A2609F4A140A6958FEF6B
:100CC000811D811D089597F99F6780E870E060E0BD
:100CD00008959FEF80EC089500240A9416161706D5
:100CE00018060906089500240A941216130614061D
:100CF00005060895092E0394000C11F4882352F080
:100D0000BB0F40F4BF2B11F460FF04C06F5F7F4F37
:100D10008F4F9F4F089557FD9058440F551F59F01E
:100D20005F3F71F04795880F97FB991F61F09F3FD8
:100D300079F087950895121613061406551FF2CF01
:100D40004695F1DF08C0161617061806991FF1CF51
:100D500086957105610508940895E894BB27662778
:100D60007727CB0197F908950E94C7060C947A065D
:100D70000E946C0638F00E94730620F0952311F053
:100D80000C9463060C94690611240C94AE060E9420
:100D90008B0670F3959FC1F3950F50E0551F629F2E
:100DA000F001729FBB27F00DB11D639FAA27F00DC4
:100DB000B11DAA1F649F6627B00DA11D661F829FEB
:100DC0002227B00DA11D621F739FB00DA11D621FD0
:100DD000839FA00D611D221F749F3327A00D611DED
:100DE000231F849F600D211D822F762F6A2F1124CF
:100DF0009F5750409AF0F1F088234AF0EE0FFF1F02
:100E0000BB1F661F771F881F91505040A9F79E3F58
:100E1000510580F00C9463060C94AE065F3FE4F33A
:100E2000983ED4F3869577956795B795F795E795AE
:100E30009F5FC1F7FE2B880F911D9695879597F9B7
:100E40000895A1E21A2EAA1BBB1BFD010DC0AA1F0B
:100E5000BB1FEE1FFF1FA217B307E407F50720F023
:100E6000A21BB30BE40BF50B661F771F881F991F9E
:100E70001A9469F760957095809590959B01AC01E7
:100E8000BD01CF010895EE0FFF1F0590F491E02DF5
:100E90000994F894FFCF000000002C018C00B900E9
:100EA0007901EA00C800DC0043757272656E742037
:100EB00068756D64697479203D20002025000D0A55
:100EC0000043757272656E742074656D7065726131
:0C0ED00074757265203D20002043000076
:107E0000112484B714BE81FFF0D085E080938100F7
:107E100082E08093C00088E18093C10086E0809377
:107E2000C20080E18093C4008EE0C9D0259A86E02C
:107E300020E33CEF91E0309385002093840096BBD3
:107E4000B09BFECF1D9AA8958150A9F7CC24DD24C4
:107E500088248394B5E0AB2EA1E19A2EF3E0BF2EE7
:107E6000A2D0813461F49FD0082FAFD0023811F036
:107E7000013811F484E001C083E08DD089C08234E0
:107E800011F484E103C0853419F485E0A6D080C0E4
:107E9000853579F488D0E82EFF2485D0082F10E0AE
:107EA000102F00270E291F29000F111F8ED06801E7
:107EB0006FC0863521F484E090D080E0DECF843638
:107EC00009F040C070D06FD0082F6DD080E0C81688
:107ED00080E7D80618F4F601B7BEE895C0E0D1E017
:107EE00062D089930C17E1F7F0E0CF16F0E7DF06D8
:107EF00018F0F601B7BEE89568D007B600FCFDCFD4
:107F0000A601A0E0B1E02C9130E011968C91119780
:107F100090E0982F8827822B932B1296FA010C0160
:107F200087BEE89511244E5F5F4FF1E0A038BF0790
:107F300051F7F601A7BEE89507B600FCFDCF97BE46
:107F4000E89526C08437B1F42ED02DD0F82E2BD052
:107F50003CD0F601EF2C8F010F5F1F4F84911BD097
:107F6000EA94F801C1F70894C11CD11CFA94CF0C13
:107F7000D11C0EC0853739F428D08EE10CD085E9AC
:107F80000AD08FE07ACF813511F488E018D01DD067
:107F900080E101D065CF982F8091C00085FFFCCF94
:107FA0009093C60008958091C00087FFFCCF809118
:107FB000C00084FD01C0A8958091C6000895E0E648
:107FC000F0E098E1908380830895EDDF803219F02E
:107FD00088E0F5DFFFCF84E1DECF1F93182FE3DFCA
:107FE0001150E9F7F2DF1F91089580E0E8DFEE27F6
:047FF000FF270994CA
:027FFE00040479
:00000001FF
